:10000000020F3C8F828E83E5821582AE83700215CB
:10001000834E60097F147E001213A380EA223232DD
:0300230002001EBA
:03002B00020FC8F9
:1000330002001FBB010689828A83F0225002F72245
:10004300BBFE01F322EF8DF0A4A8F0CF8CF0A4281F
:10005300CE8DF0A42EFE22BC000BBE0029EF8DF046
:1000630084FFADF022E4CCF875F008EF2FFFEE33F8
:10007300FEEC33FCEE9DEC984005FCEE9DFE0FD5A7
:10008300F0E9E4CEFD22EDF8F5F0EE8420D21CFE7B
:10009300ADF075F008EF2FFFED33FD4007985006E4
:1000A300D5F0F222C398FD0FD5F0EA22C2D5EC3089
:1000B300E709B2D5E4C39DFDE49CFCEE30E715B23D
:1000C300D5E4C39FFFE49EFE12005AC3E49DFDE402
:1000D3009CFC800312005A30D507C3E49FFFE49EC3
:1000E300FE22C5F0F8A3E028F0C5F0F8E5821582FA
:1000F30070021583E038F022E88FF0A4CC8BF0A4D3
:100103002CFCE98EF0A42CFC8AF0EDA42CFCEA8EE6
:10011300F0A4CDA8F08BF0A42DCC3825F0FDE98F09
:10012300F0A42CCD35F0FCEB8EF0A4FEA9F0EB8F00
:10013300F0A4CFC5F02ECD39FEE43CFCEAA42DCECD
:1001430035F0FDE43CFC2275F008758200EF2FFFCB
:10015300EE33FECD33CDCC33CCC58233C5829BED9C
:100163009AEC99E58298400CF582EE9BFEED9AFDA0
:10017300EC99FC0FD5F0D6E4CEFBE4CDFAE4CCF950
:10018300A88222B800C1B90059BA002DEC8BF084C3
:10019300CFCECDFCE5F0CBF97818EF2FFFEE33FE91
:1001A300ED33FDEC33FCEB33FB10D703994004EB49
:1001B30099FB0FD8E5E4F9FA227818EF2FFFEE3315
:1001C300FEED33FDEC33FCC933C910D7059BE99A27
:1001D3004007EC9BFCE99AF90FD8E0E4C9FAE4CCB8
:1001E300FB2275F010EF2FFFEE33FEED33FDCC3322
:1001F300CCC833C810D7079BEC9AE899400AED9B0B
:10020300FDEC9AFCE899F80FD5F0DAE4CDFBE4CCE9
:10021300FAE4C8F922E8600FECC313FCED13FDEE1A
:1002230013FEEF13FFD8F122A42582F582E5F03502
:1002330083F58322E493FB740193FA740293F92206
:10024300D083D082F8E4937012740193700DA3A34A
:1002530093F8740193F5828883E47374029368605E
:10026300EFA3A3A380DFEC8EF0A4CCC5F0CCCDF834
:10027300EFA4CEC5F02DFDE43CFCE8A42EC8C5F0E8
:100283003DFDE43CFCEFA4FFE5F028FEE43DFDE486
:100293003CFC228F358C368D37E4F543F544F5412C
:1002A300F542F538E538C3953540030203809000E5
:1002B300B5E0FF6538701CE5192FFFE412094BFC0C
:1002C300A3E0FD120936FEA3E0C39DF540EE9CF5C5
:1002D3003F8064120922120942120A0F8F3C8E3B9F
:1002E3008D3A8C39E5192538FFE412092D120A25B8
:1002F300AF3CAE3B1201868E3D8F3E12092212099E
:1003030042120A1A953EFFEE953DAB07FAE4F9F85F
:10031300AF3CAE3BAD3AAC391201868E3D8F3E9079
:1003230000B5E02519FFE412092DFEA3E0C3953EB5
:10033300F540EE953DF53FC3E53F6480948050055D
:10034300E4F53FF540D3E5409542E53F9541401440
:10035300854546854143854244853845853F4185EA
:1003630040428014D3E5409544E53F9543400985D9
:100373003846853F4385404405380202A7E54225B8
:1003830044FFE5413543FEC3EF9537EE95365005FF
:100393007EFF7FFF22E536C313FEE53713FFC3E578
:1003A300429FF540E5419EF53FFEAF407C007D0A4C
:1003B3001200481209F8EDD3941F40027D1FEDACE3
:1003C30036AD371209B4CEC313CE13D8F9F53E8E2A
:1003D3003D2542F542E53D3541F541E53E2544F5F0
:1003E30044E53D3543F543E544AE437807C333CE97
:1003F30033CED8F9FF1209F8900124E07002A3E08C
:1004030070051209D1800D120A02CEC313CE13D880
:10041300F912098A120A2FCEC313CE13D8F9FD900D
:1004230000D0E545F075F040A485F047F548E54573
:100433001209E15002AD07E545120960C333CE331B
:10044300CED8F9120972AD07AC06E545700AE53559
:1004530014B54604C206801BE53514B54508E546C8
:100463007004D206800DE545C395465004D206803C
:1004730002C20630060CED2548F548EC3547F54732
:100483008022E54845477011E53575F040A4AEF08C
:1004930024FFF548EE34FFF547C3E5489DF548E5ED
:1004A300479CF547AE47AF4822E4F532F5F875FBB4
:1004B3003FD20153D57F43D501E5F854F84407F5FE
:1004C300F853F8BF75F90F75FA329081037440F051
:1004D300E4F5E8F5C0908030F090FC00E04440F093
:1004E300E58654F04407F586E4F5161212EF75A17C
:1004F300A575D58075D67FE532601F908030E054B6
:100503007FF0E054FE4401F0C2AF438702000000D5
:10051300E04480F0E054FEF0D2AF900100E0FF121F
:10052300089F4003020637AEFBEE60CBEF60021478
:10053300F0E4FDED1208EA40030206107E007401A8
:10054300A805088005C333CE33CED8F9FFACFBEC46
:10055300FBEF5B700302060CA8057401088002C35D
:1005630033D8FCF5FBEDFF7E00700885E23385E1AF
:10057300348044EF64014E700885E43385E33480AE
:1005830036EF64024E700885E63385E5348028EF44
:1005930064034E700885D93385E734801AEF640409
:1005A3004E700885DB3385DA34800CEF64054E70BA
:1005B3000685DD3385DC34E532702CE53424F7FF22
:1005C300E53334FFFEE5162DFC1208DEEEF0A3EF53
:1005D300F0E5342409FFE43533FEEC120918F58302
:1005E300EEF0A3EFF08022E5162DFF1208DEE0FA0D
:1005F300A3E0C39534EA9533503AEF120918120871
:1006030059D39534EE9533402B0D020536E5162468
:100613000612087C500874062516F516800DE4F5BD
:1006230016E532700675320143F8201212EF75A1F8
:10063300A50204FAE4F5F875FB3FE58654F0440D92
:10064300F5861208C9908030E04440F053D57F43CB
:10065300D5017F017E001213A375D580E4F5D6F58D
:1006630016121111120911C20175E8E322C20575B0
:100673001908200307D2037F0412115F7D3A7C001F
:100683007F04120296EFF47002EEF46002C204904B
:100693000123E0F9600302077A900122E06003027C
:1006A300074AEFF47002EEF4600B7401F09000FF60
:1006B30004F00207CA85193212083A40030207CA36
:1006C30012081BE53212080FE0FAA3E0FBD39DEA00
:1006D3009CE532400712081DC3EB801412080FE09B
:1006E300FCA3E0FDE5321208A7F583E0FAA3E0C31B
:1006F3009DF534EA9CF533D3E5349408E53394004F
:10070300502174162532120832E0703612081BE5A8
:100713003212080FECF0A3EDF012081BE5321209B8
:1007230007800E12081BE53225E02402F582E4342B
:1007330000F583ECF0A3EDF0741625321208327441
:1007430032F005320206BBEFF47002EEF4600D9056
:1007530000FFE0707290012304F0806BE4900122AB
:10076300F085193212083A505E7416253212083297
:100773007432F0053280EDE96401704B900122E0A0
:100783006011EFF47002EEF4703DF09000FF74021C
:10079300F08034EFF47002EEF470269000FFE07006
:1007A30026900123F0A3F0A31208B1851932120891
:1007B3003A5014741625321208327432F00532801E
:1007C300ED9001227401F0900123E064017012EFB7
:1007D300F47002EEF4600D9000FCEEF0A3EFF080F5
:1007E300031208B29000FCE0F47003A3E0F4600489
:1007F30075180222E4F51822E53225E024B6F582C5
:10080300E43400F583E0FEA3E0FFE53225E02402B3
:10081300F582E43400F58322E53225E024B6F5823F
:10082300E43400F583E0FCA3E0FD2274162532F5E1
:1008330082E43401F58322E5192404FDE433FCC387
:10084300E5329DEC6480F874809822E53225E0243B
:10085300D1F582E43400F583E0FEA3E022740125A0
:1008630032F582E43401F58322E53275F00AA424DB
:1008730032F582E43400F58322FFE433C3FE785972
:10088300E6FDEF9D7480F86E982225E0241AF58228
:10089300E43400F583EEF0A3EFF022E0C394057493
:1008A3008094802225E024B6F582E4340022F0749B
:1008B300FF9000FCF0A3F022E53290150C93FF7833
:1008C3005BE6FEEF5E2275F90A75F84090810374CA
:1008D30057F022C39408748094802225E02428F5DD
:1008E30082E43401F58322C39406748094802278D1
:1008F30059E62401FFE433FEC32225E024D1F58227
:10090300E434002225E0241AF582E4340022900026
:10091300FB7405F02225E02440F582E434012290A3
:1009230000B5E0AD197C002DFFEC33FEEF25E0FFB1
:10093300EE33FE741A2FF58274003EF583E022FA3B
:10094300A3E0FBED2538FFEC33FEEF25E0FFEE33AC
:10095300FE74B62FF58274003EF583E022901508ED
:1009630093FCFFEDC39FFFE49400FEEF780522FFA5
:10097300ECFDC374809DFDE49400FC0200AF75F0B0
:100983000290001A02022BFFC3EB9FFFEA9E900125
:1009930024F0A3EFF0EDFF900124E48FF00200E5D3
:1009A300E5009000B675F00212022BE0FEA3E0FF13
:1009B30022FFC374209FFFE49400FE120048EF78E7
:1009C3000622C3EB9FEE6480F8EA64809822ED75FB
:1009D300F004A4FF900124E5F0F0A3EFF0229015BA
:1009E3000893FFEDC39F22E500C313FEE50013FF49
:1009F300C3E5009F22AC41AD4212005AAD072290DD
:100A03000124E0FAA3E0FBAE02780222FEA3E0FF9A
:100A1300AD03AC02020269FEA3E02BFFEE3AFEC374
:100A2300EF22FEA3E0FBAA06E4F9F822900124E0FA
:100A3300FEA3E0780222AC00AD0012005AAD0722FB
:100A4300E4F530F52FF52EF52DF53175E8E39080BB
:100A530030E04440F075A081E4F5A375A24B75A185
:100A6300A5D2AF120EB090801A7402F0C2B2121166
:100A7300DFE48F308E2FF52EF52DAD2EAC2D7808BB
:100A83001202188F1385301485140F85131012105A
:100A93004F9000FCE0FEA3E0FFF47002EEF460115F
:100AA30075310374E52FF58274133EF583E493F5F2
:100AB3004A9000FEE0604D7531031202430ADC01E7
:100AC3000AE1020AE6040AEB080AF0100AF5200A12
:100AD300FA400AFF8000000B04754A0A8026754A13
:100AE3000C8021754A0E801C754A068017754A02D0
:100AF3008012754A04800DE4F54A8008754A0F8018
:100B030003E4F5499000FEE070119000FCE0B4FFAF
:100B13000AA3E0B4FF05E4F5498003754901E549FB
:100B23007003020A91D3E5089414748094805003EF
:100B3300020A91E4F508F549F508C2AFAF31121284
:100B43008BD2AF020A91E4F532E5321208D64003A4
:100B5300020C1E12080DE0FCA3E0FD120C2F8F33D4
:100B6300E53212081D120C2F8F34EF64026007EF79
:100B730064036002C204E5337030E534701B12086D
:100B8300BB700E12082EE06003020C19EF4EF680C4
:100B93000012082E7402F0807D1208BB60691208EF
:100BA3002EE07072EFF45EF68015E534700C1207D8
:100BB300FBEEF0A3EFF0E4FD8057785BE66011E510
:100BC30032120907120806EEF0A3EFF07D0280410E
:100BD30012080DE0FEA3E0FFE53212081D7B1E7A2A
:100BE3000012131DEF602012082EE070291207FB7C
:100BF300EEF0A3EFF0E5321208A7120859FFE53231
:100C030012088D7D02800A1207FBEEF0A3EFF0AD10
:100C130034AF321213D20532020B4C785BE69000EC
:100C2300FEF0600475180122E4F51822E5329015F0
:100C33000C93785B5624FF92057B1E7A00AF321229
:100C430010B2229000B4E07015C200900100F0F5DC
:100C5300161211119000B47402F07515322290002F
:100C6300B4E064026003020D23200003020D23C2DB
:100C7300001515E5156003020D23785AF6F53212B7
:100C830008F2E5329FEE1208474003020D1FE4FF0E
:100C9300EF12089F501CE5321208FD120826E532B8
:100CA30012086E75F002EF12022BECF0A3EDF00FB9
:100CB30080DE74012532120864E4F0E53278596667
:100CC300605A12084EFFE53212088D12084EFFE5F6
:100CD3003212080FEEF0A3EFF0E5321208D6502DD2
:100CE300E53225E025E024E6F582E43414F583E4D7
:100CF30093FE740193FFE53225E024EBF582E4349F
:100D0300001208967D02AF321213D2800A741625A0
:100D1300321208327432F00532020C82784C7601BA
:100D230022908109E054E06004E044E0F0E5FB3008
:100D3300E00975FB0185E22185E122E5FB30E1094C
:100D430075FB0285E42385E324E5FB30E20975FBAB
:100D53000485E62585E526E5FB30E30975FB088573
:100D6300D92785E728E5FB30E40975FB1085DB29E6
:100D730085DA2AE5FB30E50975FB2085DD2B85DC6B
:100D83002CE4FFEF1208EA502DEF25E02421F8E6CA
:100D9300FC08E6FDE5162F1208FDF583ECF0A3ED44
:100DA300F0EFFDE5162DFDE433FC7859E66D700197
:100DB300EC60030F80CDE5162406FFE433D312085D
:100DC300804007D200E4F516800674062516F51652
:100DD300121111900100E0600214F0900127E0FF6E
:100DE300900126E0FE6F6006A3EEF075A1A522E454
:100DF300F5321208F2E5329FEE1208474003020E65
:100E0300AF120860E004F012086012089E40051259
:100E13000860E4F0C2ADE532120850FF12086CC05E
:100E230083C082120860E0D082D08375F002120280
:100E33002BEEF0A3EFF0D2ADE4F533F534F535F551
:100E43003674FFF537F538E4FFEF12089F5035127B
:100E5300086C75F002EF12022BE0FCA3E0FD2534D1
:100E6300F534EC3533F533D3ED9536EC9535400455
:100E73008C358D36C3ED9538EC953750048C378D12
:100E8300380F80C5C3E5349536FFE5339535FEC38A
:100E9300EF9538FFEE9537FE7C007D0312005AE58F
:100EA300321208A71208960532020DF522785976F8
:100EB3000CE4FFFEEEFD7C00C3940C748094805020
:100EC3002AC3ED1208D7EE501125E025E024E4F5FE
:100ED30082E43414F583740180039014FC93FDAC15
:100EE300070F744D2CF8A6050E80C9908030E0449E
:100EF30040F075D580E4F5D6D2AD1212C01208C900
:100F0300D2ADC200E49000FEF0785BF6F51812094A
:100F130011D202C201C203E4900123F09001221214
:100F230008B1E4900124F0A3F0784CF69000B4F0FB
:100F3300900127F0900126F022787FE4F6D8FD7522
:100F4300815D020F83020A43E493A3F8E493A34071
:100F530003F68001F208DFF48029E493A3F8540731
:100F6300240CC8C333C4540F4420C8834004F4562C
:100F7300800146F6DFE4800B010204081020408064
:100F830090134BE47E019360BCA3FF543F30E5090B
:100F9300541FFEE493A360010ECF54C025E060A864
:100FA30040B8E493A3FAE493A3F8E493A3C8C582F7
:100FB300C8CAC583CAF0A3C8C582C8CAC583CADF65
:100FC300E9DEE780BEC0E0C0F0C083C082C0D07558
:100FD300D000C000C001C002C003C004C005C006E9
:100FE300C007E5D530E03F43D5013001089001004B
:100FF300E004F0803C121219E51D451C6008E51D54
:10100300151D7002151C051EC3E51E948074809483
:10101300804006751E001213BDC3E50894FA748060
:10102300948050020508200108AFFBEF6003120D06
:1010330024D007D006D005D004D003D002D001D0ED
:1010430000D0D0D082D083D0F0D0E032784CE614F8
:101053006006047059020C46300042C2009001271A
:10106300E004900126F0120DF2D204E51864026048
:1010730003120B49E518640160031206703004087B
:10108300300205E58730E2031209119000FBE0709E
:101093000C3002097F01FE1200031204AC90010020
:1010A30012089E4009E4F5F875FB3F120EB0228A40
:1010B300358B36A907E9120981E0FEA3E0C39DFF42
:1010C300EE9CAB07FAE99000EB1209A830050B7C04
:1010D300007D091200480D1200AF1209C540037FBD
:1010E3000022D3EB9536E5351209C940037F01226F
:1010F300C3EA6480948040037F0222C3E49536FFF1
:10110300E49535FE1209C57F0440027F0322E4FE05
:10111300EEC394065042EEFDE5162DFDE433FC7854
:1011230059E6FBC3ED9B7480F86C98401AAF067DBB
:101133000E121253EE04FCECC39406501BAF04E4EE
:10114300FD1212530C80F0AF06E5162E244DF8E67F
:1011530004FD1212530E80B843F88022A90774FFCE
:10116300F535F536AF19E4FEE92519FDE433FCEF57
:10117300C39DEC6480F8748098502175F002EF12DF
:101183000984E0FCA3E0FDC39536EC953550099046
:1011930000B5EEF08C358D360F0E80CC228F337573
:1011A3003408D3E534940074809480402ED2B2E5A1
:1011B3003330E70D7F127E001213A3C2B27F048087
:1011C3000B7F057E001213A3C2B27F117E001213A0
:1011D300A3E53325E0F533153480C72290FC017471
:1011E30080F0E490FC06F090FC05F090FC01748123
:1011F300F0A3E0FFE48F35F534F533F532AE34ADCB
:1012030033AC3212137B121377121377F532E49057
:10121300FC01F0AC3222900000E004F0E0C394043F
:10122300748094804029E4F0FF7859E6FEEFC39E72
:10123300501574162F120832E0600974162F120825
:1012430032E014F00F80E29000FFE0600214F0221D
:10125300EF14601614601914601C14601F146022CC
:1012630024057023ED4440F5FC22ED4440F5FD22B6
:10127300ED4440F5FE22ED4440F5FF22ED4440F5F8
:10128300F122ED4440F5F2228F32D3E5329400741B
:101293008094804027D2B27F057E001213A3C2B28E
:1012A3007FB97E001213A3D2B2AF131211A0AF14F1
:1012B3001211A0AF4A1211A0153280CE2290801DC8
:1012C3007404F0E4FF7859E6FEEFC39E501D744D9D
:1012D3002FF8E675F003A42419F582E43415F58399
:1012E30012023774041200360F80DA22E4F535AFA8
:1012F30035C3EF1208EB501EE5162F12087C500B76
:10130300E5162535244DF8E6048001E4FDAF3512DA
:101313001253053580D943F88022C3EF9DFFEE9C1D
:10132300FED3EF9BEA6480F8EE6480985017C3E421
:101333009BFDE49AFCC3EF9DEC6480F8EE64809817
:1013430040037F01227F0022014900014A00014B33
:1013530000011E00010900020C0000030F00000041
:10136300010A00010E00010B000112004100000000
:1013730001150000F532FCE4FB7A01F9F81200FBD9
:101383008F358E348D338C3290FC02E0FFE5354F80
:10139300FFE534FEE533FDE5328F358E348D3322A0
:1013A300EF1FAA0670011E4A600FE4FDEDC39447C8
:1013B3007480948050EA0D80F322900100E004F0E1
:1013C300785AE66001169000FBE0600214F022ED0B
:1013D30090151493FE74162FF582E43401F583EE11
:1013E300F022101112131415161718191A1B1C1DAD
:1013F3001E1F2021222324252627282829292A2B9A
:101403002C2C2D2E2F2F30313232333435353637C5
:101413003738393A3A3B3C3D3E3E3F4040414243F8
:1014230043444546464748494A4A4B4C4C4D4E4E29
:101433004F505152535455565758595A5B5C5D5E41
:101443005F606162636465666768696A6B6C6D6E31
:101453006F707172737475767778797A7B7C7D7E21
:101463007F808182838485868788898A8B8C8D8E11
:101473008F909192939495969798999A9B9C9D9E01
:101483009FA0A1A2A3A4A5A6A7A8A9AAABACADAEF1
:10149300AFB0B1B2B3B4B5B6B7B8B9BABBBCBDBEE1
:1014A300BFC0C1C2C3C4C5C6C7C8C9CACBCCCDCED1
:1014B300CFD0D1D2D3D4D5D6D7D8D9DADBDCDDDEC1
:1014C300DFE0E1E2E3E4E5E6E7E8E9EAEBECEDEEB1
:1014D300EFF0F1F2F3F4F5F6F7F8F9FAFBFCFDFEA1
:1014E300FF000000120001000F00020028000300AB
:1014F30064000400C8000500BE00060032000700B7
:10150300280B0A090809130C1001020408102040D3
:10151300800264501E1E018019018018018007019A
:10152300800601800501800401800301800201809F
:0D1533000101800001801C01801B01801A55
:00000001FF
